:020000040000FA
:0400000004EF00F019
:080008007FEC00F067EC00F052
:10001000010EDFEC00F064EC00F0480E9FEC00F005
:10002000650E9FEC00F06C0E9FEC00F06C0E9FECE8
:1000300000F06F0E9FEC00F0200E9FEC00F0770EAA
:100040009FEC00F06F0E9FEC00F0720E9FEC00F042
:100050006C0E9FEC00F0640E9FEC00F061EC00F081
:10006000440E9FEC00F04E0E9FEC00F0300E9FEC23
:1000700000F0300E9FEC00F0330E9FEC00F0200EED
:100080009FEC00F06F0E9FEC00F06E0E9FEC00F006
:10009000200E9FEC00F0440E9FEC00F0420E9FEC0F
:1000A00000F0300E9FEC00F0310E9FEC00F0360EA9
:1000B0009FEC00F0010ED7EC00F006EF00F05FEFD0
:1000C00000F0A80EADEF00F0800EADEF00F0080ECE
:1000D000ADEC00F0010EADEC00F0C80E0DEC01F03F
:1000E000020EADEC00F0C80E0DEC01F0060EADEC0A
:1000F00000F00C0EADEC00F0C80E0DEF01F0C8ECF6
:1001000000F00A0EE7EC00F08A9A27EC01F0030EEB
:10011000BBEC00F0320E0DEC01F0030EBBEC00F076
:10012000320E0DEC01F0030EBBEC00F0320E0DECC4
:1001300001F0320EADEC00F0280EADEF00F0016ED4
:100140008A8A27EC01F001380F0BBBEC00F001505C
:10015000BBEC00F0ACEF00F01200016E8A9A27ECC5
:1001600001F001380F0BBBEC00F00150BBEC00F0CC
:10017000010EEFEF00F0026E8A8828EC01F00250C9
:1001800029EC01F08A9828EC01F0010EEFEF00F065
:10019000000E29EC01F08A9828EC01F08A9A27ECED
:1001A00001F0000E32EC01F09398939A1200016E68
:1001B0000150046E640E056E640EF7EF00F0016EE0
:1001C0000150046E640E056E140EF7EF00F0016E20
:1001D0000150046E640E056E010EF7EF00F0036E21
:1001E0000350046E0A0E056E010EF7EF00F0066E66
:1001F000FF0E076E0550096E0450086EEF0E0724BF
:10020000D8B0FFEF00F0082EFEEF00F0092EFCEF53
:1002100000F0062EFAEF00F01200016E0150026E9F
:100220000252D8B41AEF01F00A0E1BEC01F00206DC
:1002300010EF01F01200036EFF0E046E056A03500A
:100240000424D8A0000C052421EF01F012001200B4
:100250001200036E03500F0B046E8A50F00B041053
:100260008A6E1200016E01500F0B026E9350F00B5C
:060270000210936E120063
:0200000400F00A
:020000040030CA
:0E00000000260E0E00008000F0C00FE00F4042
:00000001FF
